:100000000C9496010C94BE010C94BE010C94BE019C
:100010000C94BE010C94BE010C94BE010C94BE0164
:100020000C94BE010C9424020C94B7210C9469200A
:100030000C94BE010C94BE010C94BE010C94BE0144
:100040000C943E090C94BE010C94BE010C94BE01AC
:100050000C94BE010C94BE010C94BE010C949C182F
:100060000C94BE010C945E1D0C94A11D0C94BE0159
:100070000C94BE010C94BE010C94BE010C94BE0104
:100080000C94BE010C94BE010C94BE010C94BE01F4
:100090000C94BE010C94BE010C94BE010C94BE01E4
:1000A0000C94BE010C94BE010C94BE015111571169
:1000B0005D11641172119411B211A519A8199B193F
:1000C0009F19C919C919C919AC19B019B419BA19A4
:1000D000BE19C919C419434C49206E6F742061764A
:1000E00061696C61626C652C2075736520636F6E4D
:1000F000666967757261746F72210000000002000A
:10010000080E0000030401000B00000000000000C6
:100110000000000000000000000408020110408000
:1001200040102040804080080204018040201002DE
:10013000011080102040400404040404030405025C
:100140000202020403020202020606060606060472
:100150000402020204000000002300260029002CF3
:10016000002F0000000000250028002B002E003189
:100170000000000000240027002A002D00300008A5
:100180000B0002020201000904000001020200004B
:1001900005240010010524010101042402060524A0
:1001A0000600010705810310004009040100020A4E
:1001B000000000070502024000000705830240001E
:1001C0000000C18081C112010002020000404123F1
:1001D000368000010102000112010002000000400F
:1001E0004123368000010102000118034100720022
:1001F0006400750069006E006F0020004C004C0028
:1002000043002203410072006400750069006E0023
:100210006F0020004C0065006F006E0061007200EE
:1002200064006F00040309040000000000000000E7
:100230002A2B280000000000000000000000000041
:1002400000000000000000002C9EB4A0A1A2A43475
:10025000A6A7A5AE362D3738271E1F20212223241E
:100260002526B333B62EB7B89F8485868788898ABA
:100270008B8C8D8E8F909192939495969798999A56
:100280009B9C9D2F3130A3AD350405060708090A54
:100290000B0C0D0E0F101112131415161718191A36
:1002A0001B1C1DAFB1B0B500090402000103000022
:1002B00000092101010001226500070584034000B7
:1002C0000105010902A1010901A100850105091922
:1002D000012903150025019503750181029501751A
:1002E00005810305010930093109381581257F751C
:1002F0000895038106C0C005010906A10185020514
:100300000719E029E7150025017501950881029577
:1003100001750881039506750815002565050719FF
:100320000029658100C0561B8F1E532311241FBE58
:10033000CFEFDAE0DEBFCDBF12E0A0E0B1E0E2E552
:10034000F9E402C005900D92AC32B107D9F714E080
:10035000ACE2B2E001C01D92A93EB107E1F713E0A3
:10036000CCE2D3E004C02297FE010E941C24C632D6
:10037000D107C9F70E94CB1E0C94A7240C9400004F
:1003800080910008909101088737974709F0A89558
:100390000895DC01ED91FC910190F081E02D09952B
:1003A00008958091CD03813019F482E08093CD03CC
:1003B0008091CD03833019F484E08093CD030895B8
:1003C00088E08093C10061E08AE00E94CA1960E081
:1003D0008AE00E94031A08950097C9F09C0140E04A
:1003E00050E068E478EE81E090E00E94C4232F3F63
:1003F00031054105510529F020F02FEF30E040E0B4
:1004000050E02093D1008091C000806103C08091B2
:10041000C0008F7E8093C0000895219A229A23986D
:1004200060E08BE00E94CA1961E08CE00E94CA196A
:100430000895EBE6F0E0808180688083E8E6F0E0F4
:1004400080818160808308951F920F920FB60F9272
:1004500011242F933F934F935F936F937F938F93C9
:100460009F93AF93BF93EF93FF931F9B0E94D10184
:10047000FF91EF91BF91AF919F918F917F916F917C
:100480005F914F913F912F910F900FBE0F901F9052
:100490001895A1E0B0E0EFE4F2E00C94F2231FB76E
:1004A00091E09093CC03F89489830E94C00198E175
:1004B0009093600089818093600081110E94C00147
:1004C0001FBF2196E3E00C940E2420916C03309121
:1004D0006D03382748E0C901880F991F37FF06C010
:1004E0009C0151E2252750E1352701C09C01415074
:1004F00091F730936D0320936C030895D82FC0E0DB
:10050000CD1780F45F9A64E670E080E090E00E948E
:1005100015195F9864E670E080E090E00E9415197C
:10052000CF5FEECF6CE271E080E090E00E941519A1
:10053000E6CF0F931F93CF93DF93EC01062F15E0C7
:10054000115051F0CE010E949124081741F0602F04
:10055000CE010E949924F4CF82E00E947E02DF91B6
:10056000CF911F910F910895A0E0B0E0EAEBF2E087
:100570000C94E523482E562EC0E0D0E0612C712C5F
:10058000E12CF12C00E010E041100CC06090CB0396
:1005900086E4689E30011124A9E1EA2EF12C02EBD9
:1005A00013E01EC091E049120FC06090CB03E6E457
:1005B0006E9E30011124FBE16F0E711CF9E2EF2EEB
:1005C000F12C0EE613E00CC082E0481209C078E17D
:1005D000672E77247394EE24E394F12C0BEC13E054
:1005E00043018C0E9D1E10926D0310926C0334011A
:1005F000A62CA818B12CC30101966C01AE14BF043F
:10060000A8F4A00EB11E511006C0C3010E9491248F
:10061000F501808305C0F5016081C3010E94990244
:10062000F50180810E9465023601E2CFC3015110BD
:1006300018C0C3010E949124B82EC6010E949124C3
:100640002B2D30E0322F2227282B80916C039091A4
:100650006D038217930779F4C0E0D0E055245394DA
:1006600093CF360160916D030E94990260916C03F3
:10067000C6010E949902C05EDE4FC13E92E0D907DA
:1006800008F482CF852DCDB7DEB7E0E10C940124CC
:1006900087E380936E0380E092ECA1E0B0E080936A
:1006A0006F0390937003A0937103B093720387E07C
:1006B00080937B0380E091EAACEBB3E38093730318
:1006C00090937403A0937503B093760385E08093B1
:1006D0007C038DEE9EEFADEABEED809377039093A1
:1006E0007803A0937903B0937A03EDE7F3E080E019
:1006F00090E0863028F4DC01AA50BE4F2C9101C056
:1007000020E0219301968831910599F782E080934A
:1007100095038AE080939603089561E082E00E9449
:10072000B402089560E082E00E94B4028091CB039D
:10073000843020F01092CB030E948D030895A1E035
:10074000B0E0E5EAF3E00C94F32389830E9492037E
:100750009091CB038981981731F0843020F48093F5
:10076000CB030E948D032196E2E00C940F2480E0DD
:100770009EECADEEB4E38093B3039093B403A093E7
:10078000B503B093B60380E090E0A0E0B0E58093BD
:10079000B7039093B803A093B903B093BA03EBEBFC
:1007A000F3E080E081938F5F8031E1F70895A0E06E
:1007B000B0E0EDEDF3E00C94E9230E94F21861152E
:1007C000710581059105C9F30E9488241092770371
:1007D000109278031092790310927A03C4E0C12C2E
:1007E000D12C7601CA948090770390907803A090E2
:1007F0007903B0907A03BA2CA92C982C88240E94F3
:100800008324A70196010E94C423680D791D8A1DC7
:100810009B1D609377037093780380937903909383
:100820007A03C15001F70DE713E0E801C12CD12C88
:10083000B2E38B2E912CA12CB12C80E1E82E87E223
:10084000F82E8881882309F446C0D39419F40E94B5
:10085000480341C00E948324A50194010E94C4233F
:1008600021E0260FEDE7F3E08E2F801B8C1520F49E
:1008700081918213F9CFE9CF40917C03249FA0019D
:1008800011244E9DC0014F9D900D5E9D900D112431
:10089000AA2797FDA095BA2F409173035091740336
:1008A0006091750370917603840F951FA61FB71F83
:1008B0004091B3035091B4036091B5037091B603B6
:1008C000481759076A077B0708F4BFCF2993C394D9
:1008D00088E1C812B6CFCDB7DEB7ECE00C940524A2
:1008E00061E080E00E94B40261E081E00E94B40215
:1008F000089560E080E00E94B402882331F060E057
:1009000081E00E94B402811108C00E94B7030E94D6
:1009100048030E94D7030E94700408958F929F920B
:10092000AF92BF92CF92DF92EF92FF92CF93FC01F2
:10093000C0A5EC2FE770F0E0E251FE4FA081B0E0DF
:10094000C7FF03C024E130E002C02FE030E0FC012B
:1009500097A183E1989FF0011124E25CFE4F808013
:100960009180A280B380A20FB31F20E43FE14DE746
:1009700050E00E947623A50194010E94A2238C2FAF
:10098000887149F469017A01E0EDCE0EE7E0DE1EE0
:10099000E11CF11C1BC0C7FF05C060E47AE88CE2D3
:1009A0009EE004C060E07EEE8AEB9BE069017A0184
:1009B000F8EBCF0EFBE0DF1EE11CF11CA50194015A
:1009C0000E94A223C20ED31EE41EF51EC701B6016B
:1009D00069517C4F8F4F9F4F28EE33E040E050E04D
:1009E0000E94A223A8EEB3E00E946B23CF91FF9058
:1009F000EF90DF90CF90BF90AF909F908F90089531
:100A00008F3F910551F048F0811522E0920738F0B0
:100A10008115934030F482E0089580E0089581E0EC
:100A2000089583E00895A0E0B0E0E9E1F5E00C94DA
:100A3000EE23EB018A01B82FB695A0E02881398119
:100A4000F80120832A813B8121832C813D812283EF
:100A50002E813F812383688179814A815B812C814A
:100A60003D81EE81FF819F2F9295990F990F907C88
:100A7000272F2370922B252F2370220F220F922BCA
:100A8000232F23702295207F922BF80194830B5FF4
:100A90001F4F2896AF5FBA1788F680FF24C0888161
:100AA00099810E940005D82E8A819B810E940005B1
:100AB000E82E8C819D810E940005F82E8E819F81F9
:100AC0000E940005F0E4DF9EA001112490E1E99E60
:100AD00090011124242B282BE4E0FE9EB001112468
:100AE000262BF8012083CDB7DEB7E7E00C940A246B
:100AF000803223E0920708F1883E23E0920740F419
:100B00008F519340E4E096958795EA95E1F7089533
:100B1000803D27E0920718F48C5D93400895883952
:100B200028E0920768F4885C974074E09695879572
:100B30007A95E1F78D509C4F089580E090E00895FC
:100B40008FEF93E008958C30910540F4A4E0880F76
:100B5000991FAA95E1F7885D9C4F0895843F23E093
:100B6000920718F484529C4F0895811524E092074F
:100B700040F48657934FF4E0880F991FFA95E1F7F8
:100B8000089580E998E008959C013695279525758C
:100B90003575821B930B9C01237333739695879550
:100BA0009695879583739373820F931F9C0154E0EE
:100BB000369527955A95E1F7280F391F2F703F700A
:100BC00041E051E0249FC001259F900D349F900D7E
:100BD0001124892F08952998882319F000002A9A52
:100BE00002C000002A980000299A00000895299A5E
:100BF000000083B12998000083FB882780F90895BD
:100C0000CF93DF93D82F5E9A29985E98C8E08D2FF6
:100C100080780E94EB05DD0FC150C9F72998DF915C
:100C2000CF9108958F770E9400060895CF93DF93A8
:100C3000D82FC8E08D2F80780E94EB05DD0FC150C2
:100C4000C9F72998DF91CF910895CF93DF93299821
:100C5000C8E080E0D82FDD0F0E94F7058D0FC1504E
:100C6000C9F7DF91CF9108950E9412060E942506D0
:100C70005E9A0895A1E0B0E0E0E4F6E00C94F3237E
:100C8000806869830E9400066981862F0E9416068B
:100C90005E9A2196E2E00C940F24CF93C0917703E3
:100CA000C827E82FF0E0E259FC4F678589E70E94EA
:100CB0003A066C2F8DE30E943A066C2F82E40E9464
:100CC0003A06CF91089586E20E9434060895CF93A4
:100CD000DF93EC016C818CE10E943A066D818DE11D
:100CE0000E943A066E818EE10E943A066F8180E290
:100CF0000E943A06688581E20E943A06698582E28E
:100D00000E943A066A8583E20E943A066B8584E275
:100D10000E943A066C8585E20E943A066D858AE259
:100D20000E943A066E858EE60E943A066F858FE62F
:100D30000E943A06688980E70E943A06698981E73D
:100D40000E943A066A8982E70E943A06DF91CF91B3
:100D50000895CF92DF92EF92FF92CF93DF936B01D2
:100D60007C01C11488E3D8068CE9E8068CE1F8061A
:100D700028F5C701B60120E836E948E950E00E94AD
:100D8000A223E901689760E879E687E69FEF0E9471
:100D90007E236C0D7D1D8E1D9F1DF2E0660F771F5B
:100DA000881F991FFA95D1F721E732E040E050E023
:100DB0000E94A223F22EE32E80E421C0C701B601D7
:100DC00020E03DE241E351E00E94A223E90168975F
:100DD00060E073ED8EEC9EEF0E947E236C0D7D1D16
:100DE0008E1D9F1D660F771F881F991F21E732E018
:100DF00040E050E00E94A223F22EE32E80E66C2F0A
:100E00006F71680F85E70E943A066E2D86E70E9493
:100E10003A066F2D87E70E943A06DF91CF91FF9047
:100E2000EF90DF90CF900895682F8DE60E943A06EC
:100E300008958F929F92AF92BF92CF92DF92EF92DE
:100E4000FF92CF93DF93D82F83E00E9434068093E4
:100E50006B0384E00E94340680936A0360E086E0BE
:100E60000E943A0661E087E00E943A066FE789E057
:100E70000E943A0665E08AE00E943A0665E18BE04E
:100E80000E943A0662E18CE00E943A066DEF8DE026
:100E90000E943A0660E08EE00E943A06DD2319F0D7
:100EA0008BE291E008C02091950333E1239FC001BC
:100EB0001124825C9E4F0E9467066CE880E30E94CA
:100EC0003A066FE082E30E943A0662E483E30E94FE
:100ED0003A068091960387FF02C064E101C06AE090
:100EE00084E30E943A066AE285E30E943A066DE2D4
:100EF00086E30E943A0664ED87E30E943A0660E0CA
:100F000088E30E943A0660E089E30E943A06D11124
:100F100009C0C0907703D0907803E0907903F090F7
:100F20007A0307C0C5E8CC2EC1ECDC2EED2CCEED4B
:100F3000FC2ECAE38F2C9924AA24BB24682D8C2F65
:100F40000E943A06682D85E08C0F0E943A06FE2C1E
:100F5000ED2CDC2CCC24CF5FCE3361F76FEF83E434
:100F60000E943A066FEF84E40E943A066FEF85E430
:100F70000E943A066FEF86E40E943A06DD2311F0E4
:100F800066E002C060917B038DE60E943A0660E055
:100F900089E70E943A0660917C038AE70E943A063C
:100FA00060E083E70E943A0660E084E70E943A0628
:100FB000D11109C06091730370917403809175031E
:100FC0009091760304C060E071EA8CEB93E30E9499
:100FD000A906DF91CF91FF90EF90DF90CF90BF9067
:100FE000AF909F908F90089561E087E00E943A064D
:100FF00064E28EE70E943A0663E088E00E943A06C7
:1010000060E088E00E943A0665E087E00E943A06C8
:1010100062E085E00E943A0683E00E9434068093F5
:101020006B0384E00E94340680936A03089583E092
:101030000E94340680936B0384E00E943406809300
:101040006A0361E087E00E943A066AE070E080E0AF
:1010500090E00E9415190E94F40700000895CF92B5
:10106000DF92FF920F931F93CF93DF931F92CDB721
:10107000DEB7082F162F8EE399830E943A06F02ED2
:10108000C02E9981D92E8C2D8F19811738F4F60135
:1010900061916F018FE70E943A06F5CF64E085E029
:1010A0000E943A0683E00E94340680936B0384E03A
:1010B0000E94340680936A030E94F21860936603CC
:1010C00070936703809368039093690369E087E0F6
:1010D0000E943A0681E08093CD030F90DF91CF917B
:1010E0001F910F91FF90DF90CF9008950F931F9362
:1010F0000E942F088091CD03813099F40E94F2184C
:101100000091660310916703209168033091690391
:10111000601B710B820B930B603A764881409105FE
:1011200048F38091CD03813031F467EA71E087EDB7
:1011300093E00E94FA1B1F910F9108950F931F9344
:101140008091CD03823021F41092CD0381E020C044
:101150008091CD038130D9F40E94F218009166038A
:10116000109167032091680330916903601B710B34
:10117000820B930B613A76488140910540F061E023
:1011800087E00E943A061092CD0382E001C080E021
:101190001F910F910895CF93DF93EC014AE050E047
:1011A0006D2F70E087ED93E00E94BF1C6EE287ED2B
:1011B00093E00E94CC1BBE0184E0769567958A95EA
:1011C000E1F76F7077274AE050E087ED93E00E94E7
:1011D000BF1C6EE287ED93E00E94CC1BBE016F70D6
:1011E00077274AE050E087ED93E00E94BF1CDF9133
:1011F000CF910895CF93C82F0E94F21860932A03CD
:1012000070932B0380932C0390932D03C0933F0383
:10121000CC2329F040E051EE60E070E004C040E8EB
:1012200055E260E070E089E294E00E940E1ECF91EA
:10123000089590912E03492F4F7050E0BA016F5FCF
:101240007F4F292F30E0E4E035952795EA95E1F7C7
:101250006217730759F0FA01E15DFC4F808381E06A
:10126000890F8F70907F892B80932E0308956EE7EE
:1012700070E089E294E00E94C90108951F920F92E4
:101280000FB60F9211241F932F933F934F935F93A9
:101290006F937F938F939F93AF93BF93CF93DF937E
:1012A000EF93FF93C0918600D09187008091E9026F
:1012B0009091EA0220910B03211155C09E01281B39
:1012C000390B8091B7039091B803A091B903B09105
:1012D000BA0385FD02C036952795253C49E03407C1
:1012E000B8F140910A0150E060E070E01CE1B69571
:1012F000A795979587951A95D1F70097A105B10500
:1013000021F481E090E0A0E0B0E084179507A60703
:10131000B707D8F480910A018F3FB9F040E080917F
:101320000A01481780F4842F90E0880F991FFC0170
:10133000E551FD4F20813181FC01E55FFE4F318396
:1013400020834F5FECCF10920C0310920A010BC068
:101350002D3B82E0380720F080910A018031D8F0DF
:101360008FEF80930A01D093EA02C093E902FF91C4
:10137000EF91DF91CF91BF91AF919F918F917F912D
:101380006F915F914F913F912F911F910F900FBEE1
:101390000F901F90189510910A0181E0810F8093A2
:1013A0000A01C9010E947805E12FF0E0EE0FFF1F4E
:1013B000E551FD4F91838083D6CF83E080938000F9
:1013C0008AE9809381008091B70386FD05C08091F2
:1013D00081008064809381008FEF9FEF909389005C
:1013E0008093880080916F00806280936F000895E1
:1013F0006F3018F086958058089589E0689F802D99
:1014000011240895A0E0B0E0E8E0FAE00C94ED23A8
:10141000C82F0E94F21800919A0210919B0220910D
:101420009C0230919D026B017C01C01AD10AE20A34
:10143000F30A9701860149E8C41643E1D406E104A2
:10144000F10410F010929E0260939A0270939B0236
:1014500080939C0290939D0220910B038FEF820F4B
:101460008230D8F5E0919E02EE2309F44EC1E130BE
:1014700011F482E0B8C1E03108F034C181E08E0F90
:1014800080939E02F0E0E551FD4FC083803109F06A
:10149000ACC1EDEEF2E0213029F4A181A695A6952C
:1014A000808108C080819181A92FA695A695A695D7
:1014B00096958795A03148F4B0E090E0AA0FBB1F45
:1014C000A55FBE4F11969C938E9310920C0332969B
:1014D00082E0EB3FF807F9F688C1233009F005C137
:1014E000E0919E02E11104C0CF3009F07EC10DC130
:1014F000E83148F481E08E0F80939E02F0E0E651DF
:10150000FD4FC08372C1E83109F0ECC0C111EAC0DF
:1015100040E050E0ABE0CA01B3E0880F991FBA95F4
:10152000E1F7A49F9001A59F300D1124F901E55129
:10153000FD4F6081E1817E2F777075956795FC0185
:10154000EE0FFF1FE55FFE4F71836083F901E451E9
:10155000FD4FB081B695B695B695E181FE2FF29517
:10156000FF0FF07E6F2F6B2BE695E695E6957E2FAD
:10157000777075956795FC01EE0FFF1FE35FFE4FD7
:1015800071836083F901E351FD4FB081B295B69547
:10159000B695B370C181DC2FDD0FDD0F6D2F6B2B86
:1015A000C295C695C695C370E281E170EE0FEE0F4D
:1015B0007E2F7C2B75956795FC01EE0FFF1FE15F79
:1015C000FE4F71836083F901E151FD4FB081B69503
:1015D000E181FE2FF795FF27F7956F2F6B2BE6958F
:1015E0007E2F777075956795FC01EE0FFF1FEF5EFC
:1015F000FE4F71836083F901E051FD4FB081B295D8
:10160000BF70E181FE2FF295F07F6F2F6B2BE2957B
:10161000EF707E2F777075956795FC01EE0FFF1FB9
:10162000ED5EFE4F71836083F901EF50FD4FB08195
:10163000BB1FBB27BB1FC181DC2FDD0F6D2F6B2BA9
:10164000CC1FCC27CC1FE281E370EE0F7E2F7C2BCA
:1016500075956795FC01EE0FFF1FEB5EFE4F7183E2
:101660006083F901ED50FD4FB081B695B695E181EB
:10167000FE2FF295FF0FFF0FF07C6F2F6B2BE6957F
:10168000E6957E2F777075956795FC01EE0FFF1F2D
:10169000E95EFE4F71836083F901EC50FD4F2081BC
:1016A0002295269527703181E32FEE0FEE0FEE0F76
:1016B0006E2F622B732F729576957770759567955F
:1016C000FC01EE0FFF1FE75EFE4F718360834F5FEB
:1016D0005F4F4230510509F01ECF8091010383FF17
:1016E00010920C0310929E0280C0243009F07DC03D
:1016F00060919E0261110BC0C83AB1F410926D0363
:1017000010926C0388EA0E94650281E06CC061302F
:1017100019F4C093990204C0623031F4C093980266
:101720008C2F0E9465025AC0E09198022E2F30E063
:10173000220F331F462F50E0C901029684179507E8
:101740003CF0633268F7FA01E851FD4FC083E8CFFF
:101750002D5F3F4F8C2F90E060916C0370916D0373
:101760004217530749F4982F882786279727909385
:101770006D0380936C0332C06817790769F5809117
:101780009902813049F5E13118F080E180939802A7
:10179000F0909802CCEED2E000E010E00F15D0F40B
:1017A000FE013197808190E0982F88272881822B35
:1017B00063E0969587956A95E1F70E947805F801B0
:1017C000EE0FFF1FE55FFE4F918380830F5F1F4F7A
:1017D0002296E4CF10920C0310929E0280919E02FA
:1017E000882319F08F5F80939E02CDB7DEB7E8E0C3
:1017F0000C940924E82FF0E0EE54FC4FE185E03131
:1018000058F4F894F0E0EE0FFF1FE55FFE4F2081E3
:1018100031817894C9010895E03121F0E13169F412
:1018200083E001C082E00E94361A892B19F084EF10
:1018300093E008958CE090E0089580E092E00895B0
:10184000A2E2B0E0E6E2FCE00C94E3239E012F5F0D
:101850003F4F80E1D9011D928A95E9F763EB71E072
:1018600087ED93E029A33AA30E94FA1B0E94170870
:101870001D8A1E8A1F8A188E312C212C00E0812C93
:10188000912C5401412C74E7572E7BE8672E72E3AC
:10189000772EE0E5CE2EE3ECDE2EE12CF12C84EF6A
:1018A00091E0A0E0B0E08D8F9E8FAF8FB8A380E075
:1018B0009EECADEEB4E3898F9A8FAB8FBC8F80E046
:1018C00094E7ABE8B2E3898B9A8BAB8BBC8B87ED4B
:1018D00093E00E945F1A892B09F4E1C087ED93E041
:1018E0000E94831A9C0133272C32310509F442C02F
:1018F000ACF42332310509F0ABC019821A821B8285
:101900001C821D821E821F82188619861A861B86DB
:101910001C861D861E861F86188A60C024343105E9
:1019200029F02335310509F4B2C092C064E487ED93
:1019300093E00E94CC1B2AE030E040E054E76BE8E3
:1019400072E387ED93E00E945A1C6CE287ED93E00E
:101950000E94CC1B2AE030E040E05EEC6DEE74E3C8
:1019600087ED93E00E945A1C6CE287ED93E00E94A1
:101970000C1CADCF0F5F043009F0A9CF29813A814B
:101980004B815C81A8EEB3E00E946B23698B7A8B5C
:101990008B8B9C8B2D813E814F8158850E946B23C0
:1019A000698F7A8F8B8F9C8F29853A854B855C85D3
:1019B0002D8F3E8F4F8F58A32D853E854F8558899B
:1019C0000E946B236B017C0160323EE4730781054A
:1019D000910530F462E38CE10E943A0600E077CF93
:1019E000603345E774078105910510F462E2F3CF97
:1019F00060345CE975078105910510F466E2EBCF70
:101A000080E5C81683ECD806E104F10410F462E125
:101A1000E2CF90E6C9169AEED906E104F10410F47B
:101A200065E1D9CFA0E7CA16A1E1DA06A1E0EA068E
:101A3000F10410F461E0CFCFB0EACB16B6E8DB06D4
:101A4000B1E0EB06F10410F463E0C5CF65E0C3CF6D
:101A500010ED180F1A3008F03ACFE1E0F0E0EC0F8B
:101A6000FD1F24E0029FE00DF11D11242081318132
:101A700042815381AAE0B0E00E946B23610F711D87
:101A8000811D911D608371838283938320CF498858
:101A90005A886B887C88812C912C540118CF811432
:101AA0009104A104B10489F4C301B2010E94A90602
:101AB00061E070E080E090E00E9415191D8A1E8AA6
:101AC0001F8A188E312C22242A948D8D9E8DAF8DE5
:101AD000B8A188169906AA06BB06D0F40E94630630
:101AE0002D893E894F89588D280F311D411D511D6B
:101AF0002D8B3E8B4F8B588F381608F4382E82155D
:101B000008F4282E3FEF831A930AA30AB30A56C09B
:101B1000C301B20128EE33E040E050E00E94A2236E
:101B2000BA01A9012AE030E087ED93E00E94A81CE9
:101B30006CE287ED93E00E94CC1B4AE050E0632DFD
:101B400087ED93E00E94B71C6CE287ED93E00E9462
:101B5000CC1B6D897E898F89988DA50194010E9487
:101B6000A223BA01A9012AE030E087ED93E00E94A8
:101B7000A81C6CE287ED93E00E94CC1B4AE050E089
:101B8000622D87ED93E00E94B71C6CE287ED93E035
:101B90000E940C1C4C0C5D1C6E1C7F1C898D9A8D48
:101BA000AB8DBC8D84159505A605B70520F4498835
:101BB0005A886B887C88812C912C540129893A8918
:101BC0004B895C89283E33404105510509F07FCEA1
:101BD000A296E2E10C94FF23ACE1B0E0E2EFFDE07D
:101BE0000C94ED230E94F2186B017C0181E00E94AD
:101BF000190714E703E0198361E0CE0101960E9402
:101C000076080093CD030E94F4076AEF70E080E04D
:101C100090E00E9415198091CD03833089F487EDFF
:101C200093E00E945F1A892B59F40E94F2186C19F4
:101C30007D098E099F096038734C894C9140D8F218
:101C40008091CD03833009F44FC08FE70E941206C4
:101C50000E9425068983843511F083E05CC00E94D0
:101C6000250610924003809341030E94250620918F
:101C7000400330914103280F311D309341032093DD
:101C800040030E942506809342030E94250680930C
:101C90004303813110F7F12C0F2D10E080914303A5
:101CA00090E0880F991F0817190740F40E94250635
:101CB000F801EC5BFC4F8083F394EECF80E78983DF
:101CC00061E0CE0101960E94760883E08093CD0307
:101CD0000E94F40762E370E080E090E00E94151932
:101CE0008091CD03833011F482E015C08FE70E940C
:101CF00012060E9425068983803509F0AECF07E9D8
:101D000013E00E942506F80181938F01F3E0023B66
:101D10001F07B9F781E06C96E8E00C940924CF9393
:101D2000C82F682F87ED93E00E94D01A909164032A
:101D30009C2790936403CF910895A1E0B0E0E3EA7B
:101D4000FEE00C94F32399830E948F0E9981892FD2
:101D50000E948F0E2196E2E00C940F241F93CF93E4
:101D6000DF93182FEB011092640365EB87ED93E08E
:101D70000E94D01A62E687ED93E00E94D01A812F6C
:101D80000E948F0ECE010E949D0EDF91CF911F9178
:101D900008956091640387ED93E00E94D01A08953E
:101DA000A1E2B0E0E6EDFEE00C94EF237B018A01B6
:101DB0008B3009F42EC108F03FC0853009F49BC078
:101DC00010F5823009F47EC058F4813009F030C239
:101DD00069E270E081E00E94AE0E0EE613E068C09A
:101DE000833009F480C0843009F022C261E070E0E1
:101DF00084E00E94AE0E81E00E948F0E0E94C90E08
:101E00000E94200C1FC2883009F49BC070F48630F9
:101E100009F48DC0873009F00BC261E070E087E003
:101E20000E94AE0E8091420309C2893009F491C02C
:101E30008A3009F4C3C0FCC1893609F469C178F459
:101E4000863609F41AC120F4853609F402C1F0C1BE
:101E5000873609F426C1883609F42BC1E9C18C36CE
:101E600009F49FC190F48A3609F45CC18B3609F0FD
:101E7000DFC161E070E08BE60E94AE0EF801808168
:101E80000E949F030E947904BEC18D3609F4BDC132
:101E9000873C09F0CDC161E070E087EC0E94AE0E96
:101EA00081E00E948F0E0E94C90E10926503CAC184
:101EB000F80181918F010E948F0EF3E007391F070F
:101EC000B9F7BEC16BE170E082E00E94AE0E07E997
:101ED00013E0F80181918F010E948F0EF3E0023B25
:101EE0001F07B9F7ADC161E070E083E00E94AE0E5C
:101EF0000E94EC0DA3C16091430370E0660F771F51
:101F000085E00E94AE0E04E413E08091430390E06C
:101F1000880F991F9801245433402817390708F077
:101F20008FC1F80181918F010E948F0EEECF62E088
:101F300070E086E00E94AE0E84E793E00E949D0E62
:101F40007FC161E070E088E00E94AE0E8091CB031B
:101F500075C186E6898361E0CE0101960E9476080C
:101F60000E94F40783E08093CD0368EC70E080E08A
:101F700090E00E9415198091CD038430D9F48FE749
:101F80000E9412060E9425068983863469F460E265
:101F900070E089E00E94AE0E10E20E9425060E94C9
:101FA0008F0E1150D1F74CC161E070E089E00E94C2
:101FB000AE0E29C161E070E089E03DC169E170E0E9
:101FC0008AE00E94AE0E81E08093B2032091CC03A0
:101FD0008091B7039091B803A091B903B091BA036F
:101FE000222311F0806801C08F778093B70390930C
:101FF000B803A093B903B093BA0302EB13E0F8015E
:1020000081918F010E948F0EF3E00B3C1F07B9F7FF
:1020100017C161E270E08BE00E94AE0E80910C036C
:102020008F3F39F080910C0391E0980F90930C034F
:1020300002C080910C030E948F0E10E0812F0E943D
:10204000FA0B0E94A3050E949D0E1F5F1031B1F78D
:10205000F7C061E070E085E60E94AE0E89E2E81606
:10206000F10409F0EAC0D801EEE6F3E08D91819326
:1020700083E0E739F807D1F7C6C061E070E086E693
:102080000E94AE0EEBE1EE16F10409F0D6C0D801C5
:10209000E7E9F3E08D91819383E0E23BF807D1F724
:1020A000B2C061E070E087E60E94AE0E0E9470044C
:1020B000AAC061E070E088E60E94AE0E85E78983E1
:1020C0008BE1E7E9F3E0DE01129601900D928A952B
:1020D000E1F76CE1CE0101960E9476080E94F407B8
:1020E00083E08093CD0360E273E080E090E00E94A3
:1020F00015198091CD03843009F09FC08FE70E94AD
:1021000012060E9425068983853509F096C07BC09A
:1021100061E070E089E60E94AE0E0E9448030E94D2
:10212000B70371C061E070E08AE60E94AE0E89E6F6
:10213000898361E0CE0101960E9476080E94F4072F
:1021400083E08093CD0360E273E080E090E00E9442
:1021500015198091CD03843009F06FC08FE70E947C
:1021600012060E94250689838E010E5F1F4F7E0195
:10217000EDE1EE0EF11C0E942506F80181938F011E
:10218000EE15FF05C1F78BE1FE013296A7E9B3E03A
:1021900001900D928A95E1F78981893409F04DC04B
:1021A00032C061E070E08CE60E94AE0EF0E2EF1605
:1021B000F10461F487E6898380E2F801DE0112967A
:1021C00001900D928A95E1F761E203C087E489836B
:1021D00061E0CE0101960E9476080E94F40783E038
:1021E0008093CD036CE474E080E090E00E941519C8
:1021F0008091CD03843009F58FE70E9412060E947A
:1022000025068734D1F481E019C061E070E08DE6E5
:102210000E94AE0E89E1E816F10479F4D801E2EBF0
:10222000F3E08D91819383E0EB3CF807D1F7EBCF9E
:1022300061E070E08AEC0E94AE0E80E00E948F0E9A
:102240000E94C90EA196E6E00C940B24A0E0B0E039
:10225000ECE2F1E10C94ED23CCE2D2E014E606E0EE
:1022600035E0F32E44E0E42E53E0D52E62E0C62E96
:1022700087ED93E00E945F1A892B09F49BC087EDDC
:1022800093E00E94831A282F809397024091960230
:1022900050E04730510560F7FA01EA5AFF4F0C94BD
:1022A0001A24853B29F781E080939602E1CF82369C
:1022B00009F07DC0C0929602DBCF80939502809397
:1022C0009402D0929602D4CF9C013327309393028C
:1022D0002093920290919402982790939402E09216
:1022E0009602C6CF382F2227409192025091930236
:1022F000242B352B309393022093920290919402D9
:10230000982790939402F09296022536310508F4AE
:10231000AFCF61E070E08CEC0E94AE0E81E00E94D5
:102320008F0E0E94C90E43C02091900230919102FD
:10233000F901E45DFD4F808390919402982790937A
:102340009402C9010196909391028093900220918A
:102350009202309193028217930708F489CF009379
:10236000960286CF8091940282130BC060919002F6
:10237000709191024CE252E0809195020E94D00E41
:102380000DC062E070E08BEC0E94AE0E8091950271
:102390000E948F0E809164030E948F0EFE01812F98
:1023A00011928A95E9F71092910210929002109280
:1023B00096025ECFCDB7DEB7E8E00C94092481E049
:1023C0008093650380916503882349F087ED93E04E
:1023D0000E945F1A892BB1F30E942611F3CF089552
:1023E000AAE2B0E0E6EFF1E10C94EB230E94E618DC
:1023F0006B017C0181E00E94190787ED93E00E9448
:102400005F1A892B29F087ED93E00E94831AF5CF9C
:102410005F9811E072E6B72EE9E2AE2E03E00E946B
:10242000E6186C197D098E099F09693C71058105C3
:102430009105D0F11123C1F10E94E6186B017C01D6
:10244000469A80ED97E00E94EC01B982EEE6F3E057
:10245000DE0112968A2D01900D928A95E1F76AE2CB
:10246000CE0101960E947608469880E090E00E9496
:10247000EC010093CD030E94F40762E370E080E07A
:1024800090E00E9415198091CD03843061F400938F
:10249000CD038FE70E9412060E94250611E08234C8
:1024A00019F410E001C011E082E10E94361A892B74
:1024B00081F411E00EC05F9A469A87ED93E00E9486
:1024C000831A8D309105A9F05CF40A9791F05F981A
:1024D000469887ED93E00E945F1A892B61F79FCFA2
:1024E0008332910569F08234910589F70E94DF11EA
:1024F000EECF66ED70E087ED93E00E94E81BE7CF3A
:102500000E94200CE4CF8F929F92AF92BF92CF9205
:10251000DF92EF92FF921F93CF93DF9382E10E94AD
:10252000361A892B09F078C068EC70E080E090E002
:102530000E94151980E090E00E94EC010E94E618CC
:102540004B015C016B017C0180ECC80E82E1D81E5E
:10255000E11CF11C0E94E6186C157D058E059F0597
:1025600030F482E10E94361A892BA1F353C082E134
:102570000E94361A892B09F04DC080ED97E00E9429
:10258000EC010E94E6186B017C01D0E0C1E088E418
:10259000880E86E2981EA11CB11C11E082E10E9407
:1025A000361A892B21F58C149D04AE04BF0430F437
:1025B00080ED97E00E94EC01D1E0F0CF0E94E61898
:1025C0006C197D098E099F09693C7105810591058A
:1025D00028F30E94E6186B017C01C12719F080EDF9
:1025E00097E002C080E090E00E94EC01D7CF80E04D
:1025F00090E00E94EC01DD2349F08091CB038F5FD6
:1026000083700E949F030E94790406C00E94D70332
:102610000E9470040E94F011DF91CF911F91FF90F2
:10262000EF90DF90CF90BF90AF909F908F900895E4
:10263000CF92DF92EF92FF9280E00E9449020E94C7
:102640000D0261E086E00E94CA1961E085E00E9407
:10265000CA1960E082E10E94CA1960E084E00E9429
:10266000CA1961E084E00E94031A0E94E00160E060
:1026700070E087ED93E00E94551B0E9492030E9438
:1026800079040E94DD098FEF80930C030E941902E8
:1026900078940E94E6186B017C0180910C038F3FB7
:1026A00059F40E94E6186C197D098E099F09603D56
:1026B00077408105910588F380ED97E00E94EC0159
:1026C00061E082E10E94031A5F9A87ED93E00E9425
:1026D0005F1A892B29F087ED93E00E94831AF5CFCA
:1026E00060EC71E087ED93E00E94C91B84E793E002
:1026F0000E94CB0867ED71E087ED93E00E94C91B53
:102700004AE050E066E070E087ED93E00E94901CA4
:1027100062E370E080E090E00E94151987ED93E09D
:102720000E945F1A04970CF187ED93E00E94831AD0
:1027300082349105D1F487ED93E00E94831A8E34A0
:10274000910599F487ED93E00E94831A84349105F2
:1027500061F487ED93E00E94831A819731F480E061
:1027600090E00E94EC010E94F01140916F035091A3
:1027700070036091710370917203DB01CA010197CC
:10278000A109B1090497A105B10568F440930B03B1
:10279000433029F440EA56E861E070E004C040E0CC
:1027A00052EC61E070E089E294E00E940E1E0E940B
:1027B00083125F9880E090E00E94EC010E94DD09A6
:1027C000109227038091B70383FF11C08091830388
:1027D000882351F080918A03882331F080919103FE
:1027E000882311F087E001C085E08093270380E013
:1027F0000E941907809128030E944D060E94F40749
:102800001092A1021092A00210929F02F12C8091CE
:10281000CB038F15B0F062E370E080E090E00E949F
:10282000151980ED97E00E94EC0162E370E080E012
:1028300090E00E94151980E090E00E94EC01F39472
:10284000E6CF8091960384FF08C0982F987181E0AD
:10285000983109F080E00E94FA088FE00E94490256
:10286000FF90EF90DF90CF900895EF92FF920F933B
:102870001F93CF93DF938C016EE770E089E294E0C1
:102880000E94C901E801F12CF0E2EF2E8E0188814F
:102890008D57823048F46DE770E089E294E00E9441
:1028A000C90188818E2588832196F801608189E29B
:1028B00094E00E94201DF394F9E0FF12E7CF6EE749
:1028C00070E089E294E00E94C901CDB7DEB7E6E08E
:1028D0000C940B24A9E0B0E0E0E7F4E10C94F323BE
:1028E0009091290391110EC09EEF99838A836B8387
:1028F00050E0559547954C832D83198618861F8285
:102900001E822EC040912E03842F90E0B4E0959556
:102910008795BA95E1F7242F2F7030E0821793073F
:1029200019F18DEF89831B82FE01349650E0842FCC
:1029300090E0A4E095958795AA95E1F7242F2F7054
:1029400030E08217930749F0DC01A15DBC4F8C9108
:102950008193405F5F5F563051F740932E035A8357
:10296000CE0101960E9435148091290390E00196D2
:1029700066E070E00E948E23809329032996E2E0AE
:102980000C940F24A0E0B0E0E8ECF4E10C94EC230C
:102990006C016EE770E089E294E00E94C901860153
:1029A000E12CF12CC0E0D0E030E2B32EF8016081E0
:1029B00083E8860F823078F46DE770E089E294E076
:1029C0000E94C901F80160816B2570E089E294E002
:1029D0000E94C90104C089E294E00E94201DE11414
:1029E000F10459F0F80180819E01280F311DC901C1
:1029F000C92FDD27C80FD91FDD273FEFE31AF30AE0
:102A000089E0E816F10459F028E0E216F10421F417
:102A10008C2F8095F60180870F5F1F4FC7CFCDB7F2
:102A2000DEB7E9E00C940824A9E0B0E0EAE1F5E1C2
:102A30000C94F323E82F362F8091290390E0019620
:102A400064E270E00E948E238093290358E9598341
:102A500050E15A83813089F048F08230B9F08330F8
:102A6000D9F48B8381EF8C833D8319C085E08B8300
:102A700081EF8C832F5F2D8312C08B8381EF8C833A
:102A800084E6489FA00111245D8309C084E08B8304
:102A900081EF8C83ED8303C00E94370904C0CE010F
:102AA00001960E94C2142996E2E00C940F24A2E041
:102AB000B0E0EDE5F5E10C94E823182F762E2A839B
:102AC00049830E94F2186B017C0180913F03809042
:102AD0002A0390902B03A0902C03B0902D032A8101
:102AE00049818823C1F0D701C60188199909AA092B
:102AF000BB094C015D0191EE89169EE29906A10485
:102B0000B10420F1241708F4422F202F672D812FC4
:102B10000E94141513C0D701C60188199909AA0982
:102B2000BB094C015D0191E3891695E79906A10463
:102B3000B10460F0672D812F0E946A14C0922A03AD
:102B4000D0922B03E0922C03F0922D032296EDE01D
:102B50000C940424A2E2B0E0E0EBF5E10C94E9234C
:102B60008CE00E94340681110DC06FED71E087ED9D
:102B700093E00E94FA1B5F9A80E00E9419070E946E
:102B8000F4075F9889E294E00E94C61C892B01F14A
:102B900089E294E00E94F31C90910B03992319F0B1
:102BA0000E94020AEFCF4091A00250E09A012F5FED
:102BB0003F4F2F7133276091A10270E0261737072E
:102BC00009F3FA01E555FD4F80832093A002DACF87
:102BD00080910B03811106C08091CD03843009F0F0
:102BE00094C00DC087ED93E00E945F1A892BA1F37A
:102BF00087ED93E00E94831A0E94020AF3CF0E949D
:102C0000F218611571058105910549F0609319036A
:102C100070931A0380931B0390931C030CC081E0F4
:102C200090E0A0E0B0E08093190390931A03A09382
:102C30001B03B0931C0380910F03909110038160DC
:102C40009093100380930F0383E08093CD038FE76D
:102C50000E9412060BEC12E00E942506F8018193F7
:102C60008F01F2E0043D1F07B9F72091D402809153
:102C7000CB02982F922796FF3BC090E49227909327
:102C8000D402982F98739833F1F410E0212F30E09C
:102C90008091CB02877090E0821793074CF11F5F01
:102CA00020919603812F90E0FC01E553FD4F24FF16
:102CB00004C080810E941909E9CF608189E294E013
:102CC0000E94201DE3CF8F7399F48091CC028093F2
:102CD00018038091CD02809316038091CE028093D9
:102CE00015038091D10290E090930E0380930D0321
:102CF00080919F02813019F482E080939F0280913D
:102D00009F02833011F410929F020E94F2186B010F
:102D10007C018091110390911203A0911303B09153
:102D200014030097A105B105C9F0A7019601281B5E
:102D3000390B4A0B5B0BDA01C901883B9B40A105AB
:102D4000B10560F00E94630680931703109211038F
:102D500010921203109213031092140380911D031A
:102D600090911E03A0911F03B091200346015701CB
:102D7000881A990AAA0ABB0A8EE693E00E948E047A
:102D800086169706A806B90608F4A4C0C0921D03CB
:102D9000D0921E03E0921F03F09220030E94C00114
:102DA00080910C038830A0F08091B7039091B80314
:102DB000A091B903B091BA036CE1B695A795979528
:102DC00087956A95D1F7892B8A2B8B2B09F0A7C1A0
:102DD00080910C038F5F80930C0380911903909175
:102DE0001A03A0911B03B0911C030097A105B10524
:102DF000F1F0C81AD90AEA0AFB0A8EE693E00E94AB
:102E00008E046C157D058E059F0508F002C180912A
:102E1000B70384FD04C080ED97E00E94EC0110929E
:102E2000190310921A0310921B0310921C03909125
:102E3000D402907C9093D4025091A0028091A10280
:102E400020919F02581709F401C1223009F0FEC0F9
:102E500090589093D402E0919603E770F0E0E2512D
:102E6000FE4F6081693008F0D9C0615040E04613E0
:102E7000D7C08093A10287E3840F9091D402892B5D
:102E80008093D4024093A20283E080939F02469AEB
:102E90009091270391112DC1809128030E944D0626
:102EA000E0919603E770F0E0E251FE4F608184ED1F
:102EB00092E00E942F08E0912803EF5FE09328033F
:102EC000E83109F429C1F0E0E259FC4F87858823F5
:102ED00009F422C10E949E08813069F58091960311
:102EE000887149F180910F0390911003880F991F09
:102EF0009093100380930F0383E08093CD030E948F
:102F0000F4070E94F21860931103709312038093E8
:102F1000130390931403672B682B692B61F481E0F2
:102F200090E0A0E0B0E08093110390931203A0938F
:102F30001303B09314038091960384FF1FC0809104
:102F40000F03909110038E7F0E94C405182F60918B
:102F50000D03809118030E94F809482F612F80917A
:102F6000170349A30E94F8090091CB03282F49A118
:102F700060911503809116030E9457154698809121
:102F800025038130C1F018F08230B1F1D1C082E167
:102F90000E94361A892B09F0CBC081E0809325036B
:102FA0000E94E61860932103709322038093230309
:102FB00090932403BDC082E10E94361A892B31F51B
:102FC0000E94E618C0902103D0902203E0902303D2
:102FD000F09024036C197D098E099F09693E7340A6
:102FE0008105910508F4A4C082E08093250380ED5B
:102FF00097E00E94EC019CC082E10E94361A892B66
:1030000009F496C080E090E00E94EC011092250344
:103010008FC080E090E00E94EC0109CF68E026CFED
:10302000851709F426CF4F5F242F30E090E0F90197
:10303000EC52FD4FDC01A555BD4F7C917083F90129
:10304000EE55FD4F708301968F7111CF2430B1F48E
:103050002091A20283EA92E0A5EDB2E0FC013E2FAE
:10306000381B321718F431913D93F9CF87E3820F63
:103070009091D402892B8093D40206CF80912503AE
:10308000823069F491609093D4025F9A5BEBE52EF5
:1030900053E0F52E8E010F5F1F4FB80110C05F98EF
:1030A00080919F02811103C081E080939F028091F3
:1030B0009F02833059F784E080939F02E7CFF701A6
:1030C00081917F0169A37AA30E94FA0BF801819391
:1030D00091938F0169A17AA1FBECEF16F3E0FF0653
:1030E00071F78091960345ED52E087700E941305B9
:1030F000CECE80917B03882309F4CECE2091260387
:1031000031E0320F30932603291303C010922603B7
:1031100081500E941407C0CE10922803DBCE80910C
:103120000C03883009F45F9A89E080930C03D2CEB7
:10313000A296ECE00C9405241F920F920FB60F920A
:1031400011242F933F938F939F93AF93BF938091BD
:10315000CF039091D003A091D103B091D2033091CD
:10316000CE0323E0230F2D3720F40196A11DB11DBE
:1031700005C026E8230F0296A11DB11D2093CE03A2
:103180008093CF039093D003A093D103B093D20345
:103190008091D3039091D403A091D503B091D6032D
:1031A0000196A11DB11D8093D3039093D403A093E6
:1031B000D503B093D603BF91AF919F918F913F916B
:1031C0002F910F900FBE0F901F9018952FB7F89466
:1031D0006091CF037091D0038091D1039091D2037D
:1031E0002FBF08953FB7F8948091D3039091D403F3
:1031F000A091D503B091D60326B5A89B05C02F3F5B
:1032000019F00196A11DB11D3FBF6627782F892FA8
:103210009A2F620F711D811D911D42E0660F771F6D
:10322000881F991F4A95D1F70895CF92DF92EF92A8
:10323000FF92CF93DF936B017C010E94F218EB01A8
:10324000C114D104E104F10479F00E94F2186C1B5E
:103250007D0B683E7340A0F381E0C81AD108E108F5
:10326000F108C851DC4FECCFDF91CF91FF90EF9088
:10327000DF90CF900895789484B5826084BD84B542
:10328000816084BD85B5826085BD85B5816085BD61
:10329000EEE6F0E0808181608083E1E8F0E010827A
:1032A000808182608083808181608083E0E8F0E0BB
:1032B000808181608083E1E9F0E0808182608083A9
:1032C000808181608083E0E9F0E08081816080839B
:1032D000E1ECF0E080818460808380818260808383
:1032E000808181608083E3ECF0E080818160808375
:1032F000E0ECF0E0808182608083E2ECF0E08081AD
:1033000081608083EAE7F0E080818460808380814F
:1033100082608083808181608083808180688083F7
:10332000089590E0FC013197EE30F10590F5E35AF5
:10333000FF4F0C941A24809180008F7703C08091F6
:1033400080008F7D80938000089584B58F7702C0C0
:1033500084B58F7D84BD0895809190008F7707C0DC
:10336000809190008F7D03C080919000877F809333
:10337000900008958091C0008F7703C08091C000B5
:103380008F7D8093C00008958091C200877F8093D5
:10339000C2000895CF93DF9390E0FC01E75EFE4FFB
:1033A0002491FC01E95CFE4F8491882349F190E06F
:1033B000880F991FFC01EF58FE4FA591B4918D59CC
:1033C0009E4FFC01C591D4919FB7611108C0F8943C
:1033D0008C91209582238C93888182230AC062304D
:1033E00051F4F8948C91322F309583238C938881FB
:1033F000822B888304C0F8948C91822B8C939FBF7E
:10340000DF91CF910895A1E0B0E0E9E0FAE10C94FA
:10341000F123282F30E0F901E550FF4F8491F901A5
:10342000E75EFE4F1491F901E95CFE4F0491002321
:10343000C9F0882321F069830E9491196981E02FE6
:10344000F0E0EE0FFF1FED59FE4FA591B4919FB72D
:10345000F8948C91611103C01095812301C0812BD8
:103460008C939FBF2196E4E00C940D24CF93DF93BF
:10347000282F30E0F901E550FF4F8491F901E75E14
:10348000FE4FD491F901E95CFE4FC491CC2391F039
:1034900081110E949119EC2FF0E0EE0FFF1FEB5A03
:1034A000FE4FA591B4912C912D2381E090E021F461
:1034B00080E002C080E090E0DF91CF91089580919C
:1034C0002504909126042091270430912804821B22
:1034D000930B8F739927089520912504309126042A
:1034E00080912704909128042817390749F0E0912A
:1034F0002704F0912804EB51FC4F808190E008955F
:103500008FEF9FEF0895209125043091260480913C
:1035100027049091280428173907A9F0E09127047F
:10352000F0912804EB51FC4F8081209127043091C9
:1035300028042F5F3F4F2F733327309328042093A5
:10354000270490E008958FEF9FEF0895CF93DF93C6
:10355000C0912504D09126042196CF73DD27809158
:10356000270490912804C817D90799F082E00E9497
:10357000441F8F3F2FEF920761F0E0912504F091F7
:103580002604EB51FC4F8083D0932604C09325047E
:10359000DFCFDF91CF91089583E00E948F210895BE
:1035A000A1E0B0E0E6EDFAE10C94F1238C0169832F
:1035B0008091A401882359F041E050E0BE016F5F83
:1035C0007F4F83E00E94771F181619063CF081E0B8
:1035D00090E0F8019383828380E090E02196E4E01C
:1035E0000C940D24FC0120812E5F208342E450E0E6
:1035F0006FE771E080E80E94F71F0895FC01818168
:103600009081913A59F4813209F04BC047E050E083
:103610006DE971E080E00E94F71F45C0913209F02A
:1036200040C0803239F467E070E08DE991E00E949B
:103630003B2039C0823209F034C082818093A401DA
:1036400080919D0190919E01A0919F01B091A00158
:10365000803B9440A105B10531F58091A40180FD26
:1036600012C087E797E790930108809300082BE04A
:1036700088E190E00FB6F894A895809360000FBEA3
:103680002093600010C088E10FB6F894809360002A
:10369000109260000FBEA8951092010810920008C9
:1036A00002C080E0089581E0089508951092DA0341
:1036B0001092D90388EE93E0A0E0B0E08093DB03A2
:1036C0009093DC03A093DD03B093DE0380E092E0EF
:1036D0009093D8038093D7030895A0E0B0E0E3E788
:1036E000FBE10C94ED236C017A01EB01E60EF71E71
:1036F00000E010E0CE15DF0561F06991D601ED9193
:10370000FC910190F081E02DC6010995080F191F69
:10371000F1CFC801CDB7DEB7E8E00C9409246115FC
:10372000710589F0DB010D900020E9F7AD014150F2
:103730005109461B570BDC01ED91FC910280F3818E
:10374000E02D0995089580E090E00895EF92FF92B2
:103750000F931F93CF93DF938C01FB01C0E0D0E068
:1037600064917F018FEFE81AF80A662361F0D801AF
:10377000ED91FC910190F081E02DC8010995C80FF1
:10378000D91FF701EDCFCE01CDB7DEB7E6E00C943F
:103790000B240E948F1B0895DC01ED91FC91019098
:1037A000F081E02D099508950F931F93CF93DF9338
:1037B000EC016DE00E94CC1B8C016AE0CE010E94FE
:1037C000CC1B800F911FDF91CF911F910F91089516
:1037D0000F931F93CF93DF93EC010E94A61B8C01E4
:1037E000CE010E94D41B800F911FDF91CF911F91BA
:1037F0000F9108950F931F93CF93DF93EC010E94D5
:103800008F1B8C01CE010E94D41B800F911FDF9172
:10381000CF911F910F9108950F931F93CF93DF9333
:10382000EC010E94CC1B8C01CE010E94D41B800FA6
:10383000911FDF91CF911F910F910895A1E2B0E008
:10384000E4E2FCE10C94E9237C01C42EE52FCB01DA
:10385000D22E19A221E02D1510F02AE0D22E8E01D1
:103860000F5D1F4F8D2C912CA12CB12C6C2D7E2F18
:10387000A50194010E94A2238C2DD29E80191124AF
:10388000015011098A3010F4805D01C0895CF80193
:103890008083211531054105510521F0C22EE32F0A
:1038A000CA01E4CFB801C7010E948F1BA196ECE0CA
:1038B0000C940524A0E0B0E0E0E6FCE10C94ED23DC
:1038C000EC016A017B012115310541F4E881F981A0
:1038D0000190F081E02D642F09951DC02A3031053B
:1038E000A9F477FF12C06DE20E94CC1B8C01442723
:1038F0005527BA014C195D096E097F092AE0CE01EE
:103900000E941E1C800F911F06C02AE0B701A6016D
:10391000CE010E941E1CCDB7DEB7E8E00C9409244E
:103920000F931F93CF93DF93EC019A01AB016627AE
:1039300057FD6095762F0E945A1C8C01CE010E9483
:10394000D41B800F911FDF91CF911F910F9108958C
:103950002115310549F4DC01ED91FC910190F081D4
:10396000E02D642F099508950E941E1C08959A0168
:10397000462F50E060E070E00E94A81C08959A0174
:10398000AB0160E070E00E94A81C0895FC01248552
:103990003585F901E05CFF4F80819181F901EE5B93
:1039A000FF4F20813181821B930B8F7399270895DC
:1039B000FC0184859585FC01E05CFF4F40815181CD
:1039C000FC01EE5BFF4F208131814217530741F02C
:1039D0000190F081E02DE80FF91F808190E00895BB
:1039E0008FEF9FEF0895FC0184859585FC01E05CD5
:1039F000FF4F40815181FC01EE5BFF4F20813181FF
:103A00004217530779F0A081B181A80FB91F8C919B
:103A1000208131812F5F3F4F2F73332731832083E4
:103A200090E008958FEF9FEF0895FC0181A1882316
:103A300029F0A489B5898C9186FFFBCF11A2089546
:103A4000CF93DF93FC0126853785D901A05CBF4F5A
:103A50008D919C91119701968F739927E901CE5B07
:103A6000DF4F4881598184179507D9F30D90BC9198
:103A7000A02DA20FB31F6C93A685B785A05CBF4F86
:103A800011969C938E93A689B7892C9181E090E042
:103A9000078C02C0880F991F0A94E2F7282B2C93F9
:103AA00081E081A30488F589E02D80818064808392
:103AB00081E090E0DF91CF91089508951F920F92D9
:103AC0000FB60F9211242F933F934F938F939F9391
:103AD000EF93FF938091C80082FD1CC04091CE00FF
:103AE0008091CF049091D00401968F7399272091F3
:103AF000D1043091D2048217930771F0E091CF0482
:103B0000F091D004E157FB4F40839093D004809311
:103B1000CF0402C08091CE00FF91EF919F918F91D1
:103B20004F913F912F910F900FBE0F901F901895BE
:103B300089E294E00E94C61C892B11F00E945D1D51
:103B400008951F920F920FB60F9211242F933F9357
:103B50008F939F93EF93FF9320918B0430918C046C
:103B600080918D0490918E042817390731F480914B
:103B7000C9008F7D8093C90014C0E0918D04F0913D
:103B80008E04E55BFB4F208180918D0490918E0423
:103B900001968F73992790938E0480938D042093C0
:103BA000CE00FF91EF919F918F913F912F910F90B8
:103BB0000FBE0F901F901895A0E0B0E0E2EEFDE17F
:103BC0000C94E923FC011382128288EE93E0A0E0BA
:103BD000B0E084839583A683B78382E192E09183EA
:103BE00080837587648757874687318B208B138B3B
:103BF000028BF58AE48AD78AC68AB18EA08E938E0C
:103C0000828E8F85848F8889858F8989868F8A891E
:103C1000878F8B8980A3ECE00C940524CF92DF92F0
:103C2000EF92FF92CF93DF93EC016A017B01411584
:103C300081EE580761057105F9F0EC89FD8981E095
:103C400090E008A002C0880F991F0A94E2F78083D1
:103C500060E079E08DE390E0A70196010E94A22345
:103C600021503109410951095695479537952795B6
:103C7000211580E1380798F0EC89FD89108260E811
:103C800074E88EE190E0A70196010E94A2232150E2
:103C90003109410951095695479537952795E88986
:103CA000F9893083EA89FB89208319A2EE89FF898B
:103CB000408181E090E09C010C8C02C0220F331FF8
:103CC0000A94E2F7422B4083EE89FF8940819C01F0
:103CD0000D8C02C0220F331F0A94E2F7422B40835F
:103CE000EE89FF8940819C010E8C02C0220F331F98
:103CF0000A94E2F7422B4083EE89FF8920810F8CE2
:103D000002C0880F991F0A94E2F78095822380836E
:103D1000DF91CF91FF90EF90DF90CF9008958F9239
:103D20009F92AF92BF92CF92DF92EF92FF920F934A
:103D30001F9381E08F9385E08F9387E08F9383E0DB
:103D40008F9384E08F93EEEC8E2E912CFAECAF2EB5
:103D5000B12CA9ECCA2ED12CB8ECEB2EF12C0CEC2A
:103D600010E02DEC30E04BE454E06FE874E089E2C1
:103D700094E00E94DC1D0F900F900F900F900F9019
:103D80001F910F91FF90EF90DF90CF90BF90AF9079
:103D90009F908F9008950E943B1983ED94E00E94BC
:103DA00099210E941813C8E9DDE10E94AA15209705
:103DB000E1F30E94981DF9CF615030F02091F1009D
:103DC000FC0120830196F8CF289884E68093DA04DA
:103DD00008952FB7FC012083F89467706093E90081
:103DE0000895A1E0B0E0E7EFFEE10C94F323682F23
:103DF000CE0101960E94E91E8091F20099819FBF39
:103E00002196E2E00C940F24A2E0B0E0EAE0FFE1AA
:103E10000C94F023F62E8A019091D904992311F085
:103E200057FF03C08FEF9FEF2BC0682FCE01019685
:103E30007A830E94E91E8091F20090E0A8017A81C5
:103E4000801791070CF4AC01EF2DF72FF40E84E6E8
:103E5000FE1639F028988093DA049091F10091933E
:103E6000F7CF4115510521F08091F200882321F010
:103E700089818FBFCA0104C08BE68093E800F8CF28
:103E80002296E5E00C940C24A1E0B0E0EAE4FFE126
:103E90000C94F32341E050E0BE016F5F7F4F0E941E
:103EA000041F019719F4898190E002C08FEF9FEF02
:103EB0002196E2E00C940F24A1E0B0E0E2E6FFE1FD
:103EC0000C94F323682FCE0101960E94E91E909175
:103ED000E800892F807295FF04C09091F20080E481
:103EE000891B99819FBF2196E2E00C940F24A1E0E9
:103EF000B0E0EDE7FFE10C94E523582E7B01A42E02
:103F0000952E8091D904882369F0042F152F8AEF0C
:103F1000B82E852D8072782E9AE3892E852D807497
:103F2000682E11C08FEF9FEF53C0852D0E945C1F3C
:103F3000482E81110CC0BA94A9F361E070E080E0D2
:103F400090E00E9415190115110579F737C0282F47
:103F500030E0021713070CF4402EC42CD12C0C199E
:103F60001D09652DCE0101960E94E91E772039F0CA
:103F70004A948FEF4816B1F01092F100F9CFF70193
:103F8000842D57FE07C0815058F094919093F10012
:103F90003196F9CF815020F091919093F100FACFB2
:103FA000EC0CFD1C8091E80085FF0FC00115110588
:103FB00011F461100AC089818FBFC5CF5D9884E676
:103FC0008093DB048A2D992D03C08092E800F3CF03
:103FD0002196E0E10C9401241092E9001092D8049B
:103FE0001092D7049093D6048093D5040895CF936C
:103FF000DF93FB0120E030E0DEEF24173507A1F16D
:1040000087FF02C0C49101C0C081A091D704B091C4
:10401000D8046091D5047091D604A617B707B4F4FC
:104020009091E8009570E1F39091E80092FD1EC038
:10403000C093F1006091D7047091D8046F5F7F4FF7
:104040006F737727672B11F4D093E8006091D70442
:104050007091D8046F5F7F4F7093D8046093D7043A
:104060002F5F3F4F3196C9CFC90102C08FEF9FEF3D
:10407000DF91CF910895A1E0B0E0E1E4F0E20C948B
:10408000F223162F2091E80022FFFCCF612F7983C5
:104090000E94DC1E8BEF8093E800812F7981972F9F
:1040A0002196E3E00C940E24A1E0B0E0EAE5F0E212
:1040B0000C94F3231982CE0101960E94F21ACE01CC
:1040C00001960E943322898190E02196E2E00C94CF
:1040D0000F241F920F920FB60F921124EF92FF92AE
:1040E0000F931F932F933F934F935F936F937F9300
:1040F0008F939F93AF93BF93EF93FF93CF93DF93F0
:10410000CDB7DEB76297DEBFCDBF1092E9008091D8
:10411000E80083FFE7C068E0CE010A960E94DC1E3B
:1041200082EF8093E8009A8597FF05C08091E800B0
:1041300080FFFCCF03C08EEF8093E800892F80764C
:1041400009F0B5C08B85811105C01092F100109265
:10415000F100C1C0282F2D7F213009F4BCC085306B
:1041600049F48091E80080FFFCCF8C8580688093C3
:10417000E300B1C0863009F072C02D85E888F98867
:10418000223071F580E090E02A8B0E94EC1F0E94A3
:10419000542099E08E010F5F1F4FF801392F1192C3
:1041A0003A95E9F799832A892A8391E09E8390E8DA
:1041B00098879AEF99872091D7043091D804275F88
:1041C0003F4F3C832B838D83C7010E94EC1F49E046
:1041D00050E0B80180E00E94F71F0E9454207BC08D
:1041E000C7012A8B0E94EC1F2A89223241F482E205
:1041F00090E00E943F22892B09F06DC070C02130F1
:1042000069F488899989089711F42093D4048091DE
:10421000D404882389F066EC71E016C0233009F0DD
:104220005EC08C85882359F0823061F0813009F0BE
:1042300056C06AEE71E008C068ED71E005C064E246
:1042400072E002C062E072E06115710509F447C0D6
:10425000FB01449150E080E80E94F71F3CC087308A
:1042600009F43DC0883021F481E08093F10033C02F
:10427000893089F5937099F5E2ECF1E081E021E075
:1042800096E38093E9002093EB0034913093EC00A7
:104290009093ED008F5F3196853099F78EE780938C
:1042A000EA001092EA008C858093D90414C08889B2
:1042B00099890E94EC1F8E85811105C0CE010A9656
:1042C0000E94FE1A06C0823051F4CE010A960E9466
:1042D0006122882321F08EEF8093E80003C081E201
:1042E0008093EB0062960FB6F894DEBF0FBECDBF91
:1042F000DF91CF91FF91EF91BF91AF919F918F91FE
:104300007F916F915F914F913F912F911F910F91ED
:10431000FF90EF900F900FBE0F901F901895809315
:10432000E9008091F200882319F08AE38093E80085
:1043300008951092D90481E08093D70080EA809399
:10434000D80082E189BD09B400FEFDCF61E070E0D4
:1043500080E090E00E94151980E98093D8008CE0FD
:104360008093E2001092E000559A209A08951F92DF
:104370000F920FB60F9211242F933F934F935F9399
:104380006F937F938F939F93AF93BF93EF93FF931D
:104390008091E1001092E10083FF0FC01092E900CC
:1043A00091E09093EB001092EC0092E39093ED007B
:1043B0001092D90498E09093F00082FF26C083E029
:1043C0000E948F2182E00E94F11E882321F087ED58
:1043D00093E00E94A61A8091DB04882339F0809133
:1043E000DB0481508093DB04882369F08091DA0438
:1043F000882359F08091DA0481508093DA04811186
:1044000004C0289A02C05D9AF1CFFF91EF91BF914D
:10441000AF919F918F917F916F915F914F913F915C
:104420002F910F900FBE0F901F901895FF920F9332
:104430001F93CF93DF93EC01F62EE881F98104807E
:10444000F581E02D09958C01E881F9810680F781DD
:10445000E02D6F2DCE010995C8019927CDB7DEB7A4
:10446000E5E00C940C24FC0120812F5F208349E1BE
:1044700050E068EA72E080E80E94F71F089545E680
:1044800050E061EC72E080E80E94F71F0895A1E01F
:10449000B0E0EDE4F2E20C94EF2389838B017A0122
:1044A00041E050E0BE016F5F7F4F84E00E94771FC4
:1044B000A701B80184E40E94771F2196E6E00C94DE
:1044C0000B24FC0191818081813A31F481E09130AB
:1044D00091F0933089F411C0813271F49B3021F452
:1044E00082818093A60105C09A3031F48281809345
:1044F000A50181E00895089580E00895FC011082EF
:104500000895FC011382128222E232E0318320837B
:10451000089548E050E082E00E9447220895CF933A
:10452000DF93DC01683818F0E8E7E60F25C0E62FD6
:10453000F0E067FF11C0E058F10981E090E001C0B0
:10454000880FEA95EAF714969C911497982B149685
:104550009C931497E0E010C0E85DFD4FE491EE23DA
:1045600009F440C0E7FF08C014968C91149782604C
:1045700014968C931497EF7716968C9116978E1746
:1045800041F117968C9117978E1719F118968C9107
:1045900018978E17F1F019968C9119978E17C9F00C
:1045A0001A968C911A978E17A1F01B968C911B97D7
:1045B0008E1779F080E090E0ED01C80FD91F2E81B1
:1045C000211102C0EE8305C0019686309105A1F746
:1045D00009C0BD016C5F7F4FCD010E94892281E03F
:1045E00090E008C081E090E013969C938E93129720
:1045F00080E090E0DF91CF910895683818F0E8E707
:10460000E60F25C0E62FF0E067FF12C0E058F10981
:1046100021E030E001C0220FEA95EAF72095DC01A5
:1046200014963C911497322314963C93E0E00FC00B
:10463000E85DFD4FE491EE2329F1E7FF08C0DC01BE
:1046400014962C9114972D7F14962C93EF7720E0DD
:1046500030E0EE2351F0DC01A20FB31F16964C910F
:1046600016974E1302C016961C922F5F3F4F2630AE
:10467000310579F7BC016C5F7F4F0E94892281E090
:1046800090E0089580E090E00895FC011682178282
:1046900010861186128613861482BC016C5F7F4FD0
:1046A0000E948922089588EE94E00E947E228CED7B
:1046B00094E00E9481220895A29FB001B39FC0019F
:1046C000A39F700D811D1124911DB29F700D811D3E
:1046D0001124911D08950E945C23A59F900DB49F05
:1046E000900DA49F800D911D11240895B7FF0C9487
:1046F0006B230E946B23821B930B0895DB018F9326
:104700009F930E946B23BF91AF91A29F800D911D3B
:10471000A39F900DB29F900D1124089597FB072E33
:1047200016F4009407D077FD09D00E94202407FCDE
:1047300005D03EF4909581959F4F089570956195B1
:104740007F4F0895A1E21A2EAA1BBB1BFD010DC0CD
:10475000AA1FBB1FEE1FFF1FA217B307E407F50731
:1047600020F0A21BB30BE40BF50B661F771F881F0D
:10477000991F1A9469F760957095809590959B01A3
:10478000AC01BD01CF010895052E97FB1EF40094E6
:104790000E94DB2357FD07D00E94A22307FC03D011
:1047A0004EF40C94DB2350954095309521953F4F66
:1047B0004F4F5F4F089590958095709561957F4F0D
:1047C0008F4F9F4F08952F923F924F925F926F921B
:1047D0007F928F929F92AF92BF92CF92DF92EF9291
:1047E000FF920F931F93CF93DF93CDB7DEB7CA1B12
:1047F000DB0B0FB6F894DEBF0FBECDBF09942A883D
:10480000398848885F846E847D848C849B84AA84E4
:10481000B984C884DF80EE80FD800C811B81AA8171
:10482000B981CE0FD11D0FB6F894DEBF0FBECDBF3C
:10483000ED010895EE0FFF1F0590F491E02D09940E
:10484000AA1BBB1B51E107C0AA1FBB1FA617B707B6
:1048500010F0A61BB70B881F991F5A95A9F78095D2
:104860009095BC01CD0108958F929F92AF92BF9217
:10487000CF92DF92EF92FF92CF93DF93EC016881AA
:1048800079818A819B81611571058105910521F4EA
:1048900064E279ED8BE597E02DE133EF41E050E004
:1048A0000E94C42349015A019B01AC01A7EAB1E46B
:1048B0000E946B236B017C01ACEEB4EFA501940167
:1048C0000E947923C60ED71EE81EF91EF7FE06C009
:1048D00081E0C81AD108E10880E8F80AC882D982C4
:1048E000EA82FB82C701B6019F77DF91CF91FF90EB
:1048F000EF90DF90CF90BF90AF909F908F900895F2
:104900000E943424089586E091E00E9434240895A2
:104910006093060170930701809308019093090149
:104920000895F999FECF92BD81BDF89A992780B577
:104930000895262FF999FECF1FBA92BD81BD20BDE3
:104940000FB6F894FA9AF99A0FBE01960895F89462
:02495000FFCF97
:104952000000E904200001000000FF000200020044
:104962000200020002000200020002000200020035
:10497200020002000200020002000280250000057F
:10498200400AA1204EA50020244EA52C2330C0129F
:1049920000001A400AA1204EA5001B1E27522C23FC
:1049A200308025000005400AA1204EA50020244E9B
:1049B200A52C2330004B000006400AD0009D490080
:1049C2007B289D492C233000E1000005400A450167
:1049D200D7DC03B81E0EBF00232E48E801008A4030
:1049E2000A6001555502AD1E20000023C800E100F7
:1049F2000000000000010154582074696D656F7554
:104A02007421007363616E6E6572206D6F64650060
:104A12004F70656E4C52536E672054582073746108
:104A22007274696E672000206F6E20485720006DF7
:104A32006F64756C65206C6F636B65643F00000783
:104A42000B0C10111500160A132231290000000068
:104A5200D01A6D1B5F1A831A6C1ACC1AA61A0000A0
:104A62000000201D6D1BC61CF31CD81C151D000068
:0C4A7200000016226D1B8F22FD22452340
:1070000055C000006EC000006CC000006AC00000E7
:1070100068C0000066C0000064C0000062C00000DC
:1070200060C000005EC00000F2C400005AC0000052
:1070300058C0000056C0000054C0000052C00000FC
:1070400050C0000078C000004CC000004AC00000E2
:1070500048C0000046C0000044C0000042C000001C
:1070600040C000003EC000003CC000003AC000002C
:1070700038C0000036C0000034C0000032C000003C
:1070800030C000002EC000002CC000002AC000004C
:1070900028C0000026C0000024C0000022C000005C
:1070A00020C000001EC000001CC0000011241FBE34
:1070B000CFEFDAE0DEBFCDBF11E0A0E0B1E0E2E368
:1070C000FFE702C005900D92A83AB107D9F711E089
:1070D000A8EAB1E001C01D92AE3BB107E1F78FD342
:1070E00026C78ECFF89410926F00109281001092F4
:1070F00085001092840081E085BF15BE47985D9A97
:10710000289A0C94000008952091B2013091B301A7
:107110002F5F3F4F3093B3012093B201932F37FF7E
:1071200003C08EEF831B982F990F921710F4479886
:107130000895479A08951F920F920FB60F92112447
:107140002F938F939F93EF93FF931092850010924C
:1071500084008091A8019091A901009741F00197C6
:107160009093A9018093A801892B09F45D9A8091DD
:10717000AA019091AB01009741F001979093AB0168
:107180008093AA01892B09F4289AE0E0F0E0859128
:1071900094918F5F9F4F49F08091AC019091AD0128
:1071A00001969093AD018093AC01FF91EF919F9177
:1071B0008F912F910F900FBE0F901F90189584E024
:1071C0008093E9000DC08091E8008B778093E80000
:1071D00003C08EB3882351F08091E80082FFF9CF7D
:1071E0008091E80085FFEFCF8091F1000895982FFE
:1071F00083E08093E9008091E80085FD0DC08091D7
:10720000E8008E778093E80003C08EB3882369F08E
:107210008091E80080FFF9CF9093F1005D9884E6BB
:1072200090E09093A9018093A80108954F925F92F6
:107230006F927F928F929F92AF92BF92CF92DF9286
:10724000EF92FF920F931F93CF93DF9384E080938D
:10725000E9008091E80082FF57C2289884E690E018
:107260009093AB018093AA01AADF182F853481F493
:107270008CE49DE19093AD018093AC0107B600FCD6
:10728000FDCFF999FECF81E180935700E89503C0C7
:10729000843519F494DF8DE00DC28C34E1F3803530
:1072A000D1F3843721F484E4A2DF80E003C2813685
:1072B00011F489E5FFC18134B1F481DF182F7FDF3C
:1072C00090E0880F991FAA2797FDA095BA2F312F1C
:1072D000330F20E0442737FD4095542F822B932B0A
:1072E000A42BB52BB8C1803711F483E5E3C18335F6
:1072F00049F4C0E0D1E089917ADF21E0C730D207BC
:10730000D1F7D9C1863521F481E371DF80E3D2C1A1
:10731000833731F487E86BDF85E969DF8EE1CAC125
:107320008536B9F4E0E0F0E093E085E09093570013
:10733000E89507B600FCFDCF80935700E89507B6A7
:1073400000FCFDCFE058FF4FA0E7E030FA0771F7EF
:10735000A2CF823739F4E1E0F0E089E08093570072
:107360008491A8C1863439F4E0E0F0E089E08093AC
:10737000570084919FC18E3439F4E3E0F0E089E056
:1073800080935700849196C1813539F4E2E0F0E0B2
:1073900089E08093570084918DC1823631F489E56C
:1073A00026DF80E024DF80E885C1823419F087364B
:1073B00009F0E5C01092AD011092AC0100DF082F7A
:1073C000FEDEF82EFCDE682E8554823008F071C196
:1073D000902F80E0CF2DD0E0C82BD92B10926F00DA
:1073E000173609F04BC081E180935700E895DD2402
:1073F000CC24C3943FC0E090AE01F090AF01009167
:10740000B0011091B101B6E46B16D9F4ED2DF0E0A6
:10741000EE29FF29E4918E2FEADEDD2081F082E063
:1074200090E0A0E0B0E0E80EF91E0A1F1B1FE092FA
:10743000AE01F092AF010093B0011093B101DC24D2
:1074400018C0D801C701B695A7959795879559D5C6
:10745000CEDE82E090E0A0E0B0E0E80EF91E0A1F68
:107460001B1FE092AE01F092AF010093B0011093A8
:10747000B1012197209709F0BECF7DC08090AE0169
:107480009090AF01A090B001B090B10196E4691660
:1074900009F05DC083E0F40180935700E89507B6DA
:1074A00000FCFDCF54C0F6E46F1661F5772031F192
:1074B000E090AE01F090AF010091B0011091B101E8
:1074C0007EDED82ECC24852D90E08C299D29F701D5
:1074D0000C0140925700E895112482E090E0A0E072
:1074E000B0E0E80EF91E0A1F1B1FE092AE01F092F9
:1074F000AF010093B0011093B10102C060DE582EBD
:10750000742423C0E090AE01F090AF010091B0016F
:107510001091B10116950795F794E79450DE682F06
:10752000C701F7D48091AE019091AF01A091B00155
:10753000B091B1010296A11DB11D8093AE0190934F
:10754000AF01A093B001B093B101219704C05524BD
:10755000772444244394209709F0A5CF96E4691634
:1075600041F485E0F40180935700E89507B600FCEC
:10757000FDCF8DE03CDE82E080936F009CC08334C1
:1075800071F40091AE011091AF0119DE90E021E09D
:10759000F8010C0120935700E89511247CCE833626
:1075A00019F5E090AE01F090AF010091B00110919B
:1075B000B10105DEF701E16090E021E00C012093CC
:1075C0005700E895112482E090E0A0E0B0E0E80EDA
:1075D000F91E0A1F1B1FE092AE01F092AF0100934B
:1075E000B0011093B10157CE8D3661F4E091AE0138
:1075F000F091AF0185E080935700E89507B600FC55
:10760000FDCF49CE823551F4E091AE01F091AF014A
:1076100005911491812FEBDD802F4CC0843421F52E
:10762000E090AE01F090AF010091B0011091B10176
:1076300016950795F794E794C2DD682FC70169D4C2
:107640008091AE019091AF01A091B001B091B101D4
:107650000296A11DB11D8093AE019093AF01A0933E
:10766000B001B093B10117CE843609F5E090AE01B8
:10767000F090AF010091B0011091B101D801C701A4
:10768000B695A795979587953CD4B1DD82E090E0BB
:10769000A0E0B0E0E80EF91E0A1F1B1FE092AE0149
:1076A000F092AF010093B0011093B10104C08B318F
:1076B00011F08FE39CDD83E08093E9009091E80076
:1076C0008091E8008E778093E80095FF04C010C099
:1076D0008EB38823C9F08091E80080FFF9CF8091B4
:1076E000E8008E778093E80003C08EB3882361F0B2
:1076F0008091E80080FFF9CF84E08093E9008091D9
:10770000E8008B778093E800DF91CF911F910F9174
:10771000FF90EF90DF90CF90BF90AF909F908F90B1
:107720007F906F905F904F9008959091B601892F50
:107730008F77813249F58091B7018032A1F0813293
:1077400019F5913A09F58091E800877F8093E80068
:107750008DE091E067E070E00BD28091E8008B77DC
:107760008093E8000895913279F48091E800877F52
:107770008093E8008DE091E067E070E05DD2809159
:10778000E8008E778093E800089582E061EC42E0A3
:10779000B5D083E061E842E1B1D084E060E842E145
:1077A000ADC084B7877F84BF88E10FB6F89480931B
:1077B0006000109260000FBE20E880E090E00FB6FD
:1077C000F89420936100809361000FBE81E085BF33
:1077D00092E095BF3F9A209A559AE1E6F0E0208327
:1077E000108247985D9A289A109289008AEF8093B8
:1077F000880090936F0083E080938100F0C04091F7
:10780000000850910108109201081092000894B7E6
:1078100014BE88E10FB6F894809360001092600067
:107820000FBE292F30E0F901E270F07091FD18C011
:1078300090FF05C0859194918F5F9F4F81F423FF46
:107840000FC08091090190910A014817590741F032
:10785000E0E0F0E0859194918F5F9F4F09F042DC6A
:10786000A0DF78941092AD011092AC010CC0DEDC68
:1078700036D38091AC019091AD0181549F4110F0BD
:107880001092140141DC80911401882381F78091CA
:10789000E00081608093E00025DC80E090E00895C6
:1078A000FA01923049F0933061F09130F9F485E1BA
:1078B00091E022E130E01EC087E291E02EE330E06B
:1078C00019C0882329F485E691E024E030E012C055
:1078D000813029F489E691E022E230E00BC0823069
:1078E00029F48DE891E028E130E004C080E090E0E8
:1078F00020E030E091838083C90108958093E900FE
:107900008091EB0081608093EB001092ED0060931A
:10791000EC004093ED008091EE00881F8827881FBF
:1079200008958091B60188238CF403C08EB3882318
:10793000B1F08091E80082FFF9CF8091E8008B7769
:107940008093E80008958EB3882349F08091E80081
:1079500080FFF9CF8091E8008E778093E80008954A
:10796000EF92FF920F931F9345D04CD008ED10E09B
:10797000F80180818F778083808180688083808117
:107980008F7D808319BC1EBA1092B40180EEE82E60
:10799000F12CF70180818B7F8083F80180818160E9
:1079A000808380E060E042E0A9DFE1EEF0E08081EA
:1079B0008E7F8083E2EEF0E0808181608083808131
:1079C00088608083F70180818E7F8083F8018081C9
:1079D000806180831F910F91FF90EF900895E7EDF4
:1079E000F0E08081816080838AE482BF81E08093BF
:1079F000B501B6CFE8EDF0E080818E7F80831092F4
:107A0000E20008951092DA001092E10008951F92AA
:107A10000F920FB60F9211242F933F934F935F93C2
:107A20006F937F938F939F93AF93BF93EF93FF9346
:107A30008091DA0080FF1BC08091D80080FF17C0C2
:107A40008091DA008E7F8093DA008091D90080FFE8
:107A50000BC080E189BD82E189BD09B400FEFDCF84
:107A600081E08EBB3BD203C019BC1EBA37D28091D5
:107A7000E10080FF17C08091E20080FF13C0809179
:107A8000E2008E7F8093E2008091E200806180932B
:107A9000E2008091D80080628093D80019BC85E014
:107AA0008EBB1CD28091E10084FF2CC08091E2004B
:107AB00084FF28C080E189BD82E189BD09B400FE50
:107AC000FDCF8091D8008F7D8093D8008091E10018
:107AD0008F7E8093E1008091E2008F7E8093E200B0
:107AE0008091E20081608093E2008091B40188235C
:107AF00031F48091E30087FD02C081E001C084E0A1
:107B00008EBBECD18091E10083FF21C08091E20027
:107B100083FF1DC08091E100877F8093E10082E0B8
:107B20008EBB1092B4018091E1008E7F8093E100C2
:107B30008091E2008E7F8093E2008091E20080617C
:107B40008093E20080E060E042E0D8DEC7D1FF91A0
:107B5000EF91BF91AF919F918F917F916F915F91C5
:107B60004F913F912F910F900FBE0F901F9018953E
:107B70009C014091BC015091BD014617570718F474
:107B8000F90190E044C06115710511F0AB01F8CF27
:107B90008091E8008E778093E80040E050E0F0CFDD
:107BA0008EB3882309F444C0853009F443C0809122
:107BB000E80083FF02C081E008958091E80082FD23
:107BC00031C08091E80080FF22C08091F300909145
:107BD000F200782F60E0292F30E0262B372B07C0EA
:107BE00081918093F100415050402F5F3F4F4115EC
:107BF000510519F02830310598F390E0283031050F
:107C000009F491E08091E8008E778093E8004115B7
:107C1000510531F6992321F605C08EB3882341F032
:107C2000853041F08091E80082FFF7CF80E0089531
:107C300082E0089583E008959C016115710529F49F
:107C40008091E8008B778093E800F90126C08EB31D
:107C5000882391F1853091F18091E80083FF02C083
:107C600081E008958091E80082FFF1CF06C0809105
:107C7000F10081936150704059F02091F3008091A0
:107C8000F200322F20E090E0822B932B892B79F7A2
:107C90008091E8008B778093E80061157105B9F653
:107CA00005C08EB3882341F0853041F08091E80013
:107CB00080FFF7CF80E0089582E0089583E0089583
:107CC0000F931F93DF93CF9300D0CDB7DEB7E6EBD2
:107CD000F1E08091F100819381E0EE3BF807C9F774
:107CE00024DD8091E80083FFE4C08091B60190918B
:107CF000B701953009F46DC0963040F4913081F1B0
:107D0000913070F0933009F0D4C02AC0983009F453
:107D1000A3C0993009F4B2C0963009F0CAC07CC043
:107D2000803809F4C6C0823809F0C3C08091BA0116
:107D300087708093E9008091EB001092E900209118
:107D4000E800277F2093E80090E025E0969587954E
:107D50002A95E1F781708093F1001092F10087C0BD
:107D6000882319F0823009F0A4C08F71823009F0A5
:107D7000A0C08091B801882331F52091BA01277005
:107D800009F497C02093E9008091EB0080FF1BC0AD
:107D9000933021F48091EB00806213C08091EB005E
:107DA00080618093EB0081E090E002C0880F991F12
:107DB0002A95E2F78093EA001092EA008091EB00A6
:107DC00088608093EB001092E9008091E800877F43
:107DD00051C0882309F06DC01091B8011F770FB70B
:107DE000F8948091E800877F8093E8009ADD809185
:107DF000E80080FFFCCF8091E3008078812B8093A6
:107E0000E30080688093E300112311F482E001C055
:107E100083E08EBB0FBF4DC08058823008F049C050
:107E20008091B8019091B9016091BA01AE014F5FA4
:107E30005F4F36DDBC01009709F43BC08091E8003C
:107E4000877F8093E80089819A8192DE8091E800A3
:107E50008B778093E8002DC0803859F58091E80039
:107E6000877F8093E8008091B4018093F100809136
:107E7000E8008E778093E80054DD1BC08823C9F4A6
:107E80009091B8019230A8F48091E800877F8093A8
:107E9000E8009093B40145DD8091B401882331F46A
:107EA0008091E30087FD02C081E001C084E08EBBC9
:107EB0006CDC8091E80083FF0AC08091EB00806257
:107EC0008093EB008091E800877F8093E8000F901B
:107ED0000F90CF91DF911F910F91089508951F93F7
:107EE0008EB3882361F01091E9001092E90080912F
:107EF000E80083FF01C0E4DE17701093E9001F91D2
:107F00000895F999FECF92BD81BDF89A992780B561
:107F10000895262FF999FECF1FBA92BD81BD20BDCD
:107F20000FB6F894FA9AF99A0FBE01960895F8944C
:107F3000FFCF4341544552494E4100777700080036
:107F400000000000000801120110010200000841B9
:107F500023360001000201000109023E0002010077
:107F60008032090400000102020100052400100112
:107F7000042402040524060001070582030800FF0B
:107F800009040100020A00000007050402100001B4
:107F90000705830210000104030904220341007253
:107FA000006400750069006E006F0020004C0065E1
:107FB000006F006E006100720064006F0000001826
:107FC00003410072006400750069006E006F0020BC
:0A7FD000004C004C004300000000CC
:00000001FF
